:020000040000FA
:060000006EEF13F0120088
:060800006EEF13F0120080
:06082A000100542700004C
:0808300060000000260000003A
:0808380058EC09F0FB0EDBCFC8
:10084000F3FFDB06F35000090AE0A6EC09F0FA0E0C
:1008500011EC0AF0F3E1151CF1E1010E01D0000EDC
:1008600087EF09F058EC09F03B0EE12402E3E16860
:10087000E652E16E010EDB6A020EDB6AF90EDBCF97
:10088000F6FFFA0EDBCFF7FFFB0EDBCFF8FF080019
:10089000F550DF6EDF5002E1ABEF08F0250EDF5CB4
:1008A00002E09EEF08F0030EDB6A040EDB6A050E21
:1008B000DB6A060EDB6A070EDB6AC0EC08F02D0E61
:1008C000DF5C0CE02B0EDF5C09E0200EDF5C06E055
:1008D000230EDF5C03E0300EDF5C1AE1DF50300AEC
:1008E00014E0130A0FE0030A0AE00B0A05E0060A07
:1008F000E4E1030EDB80E1D7030EDB82DED7030EDB
:10090000DB84DBD7030EDB86D8D7030EDB88D5D795
:100910002A0EDF5C1BE1BCEC08F00AEC09F010E0E9
:10092000030EDB8006680768130EDBCF0BF0140E96
:10093000DBCF0CF099EC11F0040E04C0DBFF03D008
:10094000130EF3EC08F0C0EC08F00BD0090EDB6AD4
:1009500061EC09F003E0D5EC09F0FAD7090EF3ECED
:1009600008F0030EDBB0DB982E0EDF5C1BE1C0EC61
:1009700008F02A0EDF5C0BE1BCEC08F00AEC09F091
:1009800003E1130E45EC09F0C0EC08F00BD0090EA2
:10099000DB6A61EC09F003E0D5EC09F0FAD7090E47
:1009A00045EC09F0680EDF5C07E1C0EC08F0680E6A
:1009B000DF5C1DE1030E18D0740EDF5C17E07A0EC9
:1009C000DF5C14E0480EDF5C06E0540EDF5C03E001
:1009D0005A0EDF5C02E1020E07D06C0EDF5C03E012
:1009E0006A0EDF5C04E1010E98EC09F0C9DBDF5010
:1009F0006E0A01E17FD31E0A01E192D1200A01E1D2
:100A00008FD13F0A01E149D11A0A01E146D10D0A0D
:100A100001E143D1200A01E140D13A0A01E13DD18F
:100A2000200A01E13AD1260A01E135D10D0A01E19E
:100A300032D11A0A01E1D9D0200A4AE0300A1FE077
:100A4000460A0EE0250A01E083D3D950F90FE96E7A
:100A5000FF0EDA20EA6E010EEE5E000EEE5AEE5A3E
:100A6000A6EC09F0250EE66E95DB03E1151C01E10D
:100A700069D3A2EC09F001E26BD3DB2A69D3080E3B
:100A8000DB6A040EDB50010806E2040EDB046AECAC
:100A900009F0DB508BDB080EDB5009E0030EDB5066
:100AA000010B05E172DB01E04DD3080EDB6A64DB6C
:100AB000EFCFDFFF1AEC0AF003E1151C01E142D38E
:100AC000A2EC09F001E3DB2A60DB01E141D33AD378
:100AD000070EDB5002080FE1E6EC09F0030EADEC67
:100AE00009F00E0EEECFDBFF0F0EEECFDBFF100E88
:100AF000EECFDBFF20D0F70EDBCF17F0F80EDBCF09
:100B000018F0020E175E000E185AF70E17C0DBFF22
:100B1000F80E18C0DBFF17C0E9FF18C0EAFF9DEC14
:100B200009F0166A0E0E14C0DBFF0F0E15C0DBFFB6
:100B3000100E16C0DBFF0E0EDBCFE6FF0F0EDBCF75
:100B4000E6FF100EDBCFE6FFF3EC12F0E552E552C4
:100B5000E552130E05C0DBFF140E06C0DBFF060EC8
:100B6000DB5005E0130EE1EC09F001E26ADB05EC75
:100B70000AF002E2130E37DBC8EC09F006E0040EBF
:100B8000E1EC09F002E2050E2EDB030EDBB005D02E
:100B9000FCDA01E0D7D2080EDB6A090EDB6A0E0E22
:100BA000DBCFF6FF0F0EDBCFF7FF100EDBCFF8FF2A
:100BB0000800F550DF6EDF5014E00BEC0AF011E294
:100BC0001AEC0AF003E1151C01E1BCD2BBDB01E326
:100BD000DB2A090EDB2AD9500E0FE96E000ECBDBA3
:100BE000E7D7D3DA01E1B4D2ADD2C6DA110EEECF37
:100BF000DBFF120EEDCFDBFF110EDBCFE6FF120E97
:100C0000DBCFE6FFE5EC12F0E552E552130EF3CF31
:100C1000DBFF140EF4CFDBFF060EDB5004E0130EF7
:100C2000D0DB01E20EDB05EC0AF002E2130EDBDAA8
:100C3000AFDB05E0040EC5DB02E2050ED4DA030EDD
:100C4000DBB005D0A2DA01E07DD2080EDB6A090E26
:100C5000DB6A110EDBCFE9FF120EDBCFEAFFEFCF2D
:100C6000DFFFDF5014E0D7DB12E2E4DB03E1151C09
:100C700001E168D267DB01E3DB2A090EDB2A110EF2
:100C8000DB2ADBCFE9FF120EE8E3DB2AE6D77DDAC9
:100C900001E15ED257D2030EDB8E070EDB0410E1BA
:100CA00095DB040E5ADB0A0EEECFDBFF0B0EEECF08
:100CB000DBFF0C0EEECFDBFF0D0EEECFDBFF6CD0BB
:100CC000070EDB5003082CE1030EDBAE0DD0B2DAC9
:100CD000020E76DAEFCF14F0156A166A176A14AEB0
:100CE00039D01568166835D0F70EDBCF15F0F80E41
:100CF000DBCF16F0020E155E000E165AF70E15C069
:100D0000DBFFF80E16C0DBFF15C0E9FF16C0EAFFD7
:100D1000EFCF14F00A0E14C0DBFF0B0EDB6A38D0E5
:100D2000070EDB50020809E1030EDBAE04D059DBED
:100D300016AE10D00ED055DB0DD0030EDBAE12D0A8
:100D400079DA020E3DDAF9DA166A176A15AE02D0C0
:100D500016681768E2DA0C0E16C0DBFF0D0E17C01E
:100D6000DBFF1AD0F70EDBCF16F0F80EDBCF17F053
:100D7000020E165E000E175AF70E16C0DBFFF80EB5
:100D800017C0DBFF16C0E9FF17C0EAFFD6DAC5DAE5
:100D90000C0EDB6A0D0EDB6A060EDB5005E1010E60
:100DA000F36E050EF3CFDBFF150EDB6A160EDB6A62
:100DB000D950370F146E000EDA20156E390E14C09C
:100DC000DBFF3A0E15C0DBFF380EDB6A080EDB6A6C
:100DD0000A0EAEDADF50780A12E0200A10E0280A84
:100DE0000CE0200A0AE03F0A06E00D0A02E0200AB1
:100DF00008E1020E05D0080E03D0080EDF26100E03
:100E000097DA030EDBBE02D0DB92DB94DB50800B63
:100E100024E08ADAD890030EEB50000A08E6000EB0
:100E2000EE5C000EEE58000EEE58000EEE5815E285
:100E300013DA09680A680B680C68ADEC12F00A0E48
:100E400000C0DBFF0B0E01C0DBFF0C0E02C0DBFF9E
:100E50000D0E03C0DBFF2D0E08D0030EDBA202D067
:100E60002B0E03D0DBA408D0200EF36E170EF3CFA9
:100E7000DBFF150EDB2A02D0170EDB6A050EDB50F6
:100E800003E1B7D901E189D03E0E146E270E156E2D
:100E9000000E166E070EDBCF17F0186A196A1A6A71
:100EA00017C009F018C00AF019C00BF01AC00CF0F6
:100EB000D3D918EC13F014500024F36E1550012010
:100EC000F46E16500220F86EF4CFF7FFF3CFF6FF62
:100ED0000800090EF5CFDBFF580EDF5C0FE1610E55
:100EE000F36E090E7BD90AE3200E146E090EDBCFD8
:100EF000E7FF1450E75E090EE7CFDBFF070EDBCFFD
:100F000014F0156A166A176A0FDA14C009F015C0D2
:100F10000AF016C00BF017C00CF0EECF04F0EECFC5
:100F200005F0EECF06F0EFCF07F018EC13F007C096
:100F3000EDFF06C0EDFF05C0EDFF04C0EFFF390E69
:100F4000DBCFE9FFDB063A0EDBCFEAFF01E2DB068F
:100F5000090EDBCFEFFF150EDB2A4BD995E1030E0F
:100F6000DBA61DD06F0EDF5C06E1C1D918E3150EBC
:100F7000DB285BDA14D0780EDF5C09E0580EDF5C0A
:100F800006E0620EDF5C03E0420EDF5C08E1020E69
:100F9000F36E160EF3CFDBFF02D0150EDB6A030EE5
:100FA000DB50100B0EE0040EDBCF14F0050EDB500F
:100FB000D880145406E2060EDB5003E1040EDB5029
:100FC00034DA95D90AE2050EDBCFE7FF150EDB50C8
:100FD000E75E050EE7CFDBFF02D0050EDB6A040EED
:100FE000DBCF14F0160E45D9D880145414E2160E37
:100FF000DBCFE6FF150EDBCFE6FF040EDBCFE6FF0F
:10100000050EDB50E552E75CE552D880E754E55227
:10101000D880E7545FD9030EDB50010B0BE1080EBB
:10102000DB5008E0B2D801E08DD0080EDB50BED80E
:10103000080EDB6A170EDB5007E088D9170EF1D9CE
:1010400003E1151C01E17ED0160EDB5016E07ED9BF
:10105000300EE66E9FD802E1151C74E077D9DFCF21
:10106000E6FF6BEC12F0E552E552E552F4CF15F0D5
:101070000001F31C02E1151C65E0050EDBCF14F046
:10108000160EDB50D880145409E2050EDBCFE7FFC3
:10109000160EDB50E75E050EE7CFDBFF300EE66E87
:1010A000050ECBD94FE1390EDB2ADBCFE9FF3A0E33
:1010B00001E3DB2ADBCFEAFF090EEFCFDBFFDB50DA
:1010C0000EE044D9090EADD902E1151C3BE0390E02
:1010D000DB2ADBCFE9FF3A0EEDE3DB2AEBD755D86D
:1010E00031E1160EDBCFE6FF080EC3D8E552E72448
:1010F0005DD82ED0070EDB50030A1CE0010A14E075
:10110000030A07E07BD9DBCFEEFF020EDBCFEDFF5A
:101110001FD0F5D8196A17AE02D0186819682CD8F4
:10112000BCD819C0EEFF14D0EAD817BE186824D86E
:10113000B4D80ED063D9DBCFEFFF0AD07BD905E15D
:10114000151C03E1F368F46810D0FCD801E3DB2A36
:1011500079D947EF04F0010EDBCF14F0020EDBCF9C
:1011600015F014C0F3FF15C0F4FF3B0EE15C02E282
:10117000E16AE552E16ECBD029D9020EADEF09F05C
:1011800061D90800F550DF6E1200200EE66E080EE1
:101190001DEF0AF06BEC12F0E552E552E552F3CF89
:1011A00014F0F4CF15F00001F31C1200146E156A50
:1011B000D950010F4DD91450EE261550ED221200D2
:1011C000185E000E195AF70E18C0DBFFF80E19C092
:1011D000DBFF18C0E9FF19C0EAFF1200DBCFF4FF04
:1011E000F350F45C1200DB50E76E040EE7CFDBFF38
:1011F00012000A0EDBCF14F00B0EDBCF15F00C0E35
:10120000DBCF16F00D0EDBCF17F0145015101610B3
:1012100017101200130EEECFDBFF140EEDCFDBFF25
:10122000130EDBCF14F0140EDBCF15F00001800E8F
:1012300015141200F70EDBCF18F0F80EDBCF19F003
:101240001200050EDB50E66ED950130F01D9E5529E
:10125000E750EE6EED6A12000A0EDBCF04F00B0EC3
:10126000DBCF05F00C0EDBCF06F00D0EDBCF07F069
:101270001200DBCFE6FF150EDBCFE6FF050EDB50DD
:10128000E552E724E552E7241200DB50CED8010EE8
:10129000F36E060EF3CFDBFF1200EE50EFCFEAFF46
:1012A000E96E16C0EEFF17C0EEFF18C0EEFF120089
:1012B000D9CFE6FFDACFE6FFE1CFD9FFE2CFDAFF01
:1012C0001200DFCFE6FFE66A3CEC13F0E552E55290
:1012D000F3501200E76E080EE7CFDBFF1200EECFEF
:1012E00014F0EECF15F0EFCF16F0176A1200050ECE
:1012F000DBCF14F0150EDB50D88014541200010E11
:10130000DBCF16F0020EDBCF17F0186A1200E552A1
:10131000E5CFDAFFE7CFD9FF12000A0E14C0DBFFDA
:101320000B0E15C0DBFF1200D9500A0F28EF0AF090
:10133000F36E070EF3CFDBFF1200EECF14F0EFCF0A
:1013400015F01200010EDB2A020E1200FC0EDBCF9C
:10135000E6FFFD0EDBCFE6FF1200145E000E155A0D
:10136000F70E14C0DBFFF80E15C0DBFF14C0E9FF59
:1013700015C0EAFF1200DA20EA6EEF2AEECFF6FF80
:10138000000EEF22EECFF7FFEF22EECFF8FF1200B4
:10139000040EDBCFE6FF130EDB50E552E75C9ADF6D
:1013A000DB5004DF060EDB501200090EDB500A0D85
:1013B000F350DF24D00FE76E090EE7CFDBFFC0EF5D
:1013C00008F0DB50F36E050EEEEF08F0F70EDBCF02
:1013D00014F0F80EDBCF15F01200DFCFE6FFCAEFF6
:1013E00008F028DF030EECDE6FEF09F01CEC04F0D0
:1013F000E552E552E552E55200091200BDDEEE501D
:10140000EFCFEAFFE96E010E1200130EDB50F36E10
:10141000040EEEEF08F0040EDB50F36E090EEEEF53
:1014200008F0DBCFE6FFCAEF08F0E76E050EE7CF66
:10143000DBFF12008BDFEDEF09F0DBCFE6FF86DF8D
:10144000F6EF09F0D950F90FE96EFF0EBBEF09F086
:0A145000E96E000EDA20EA6E1200C9
:06145A00D9CFE6FFE1CF4F
:10146000D9FF040EE126DE6ADE6ADE6ADD6ADD523D
:10147000DD52FD0EDBCF14F0FE0EDBCF15F0166A49
:10148000176A15AE02D016681768D9CFE9FFDACF10
:10149000EAFF030EEB501718E8AE02D0173408D05D
:1014A0001450EE5C1550EE581650EE581750EE588A
:1014B0000FE20C0EE66E4EEC13F0E552D9CFE9FFC9
:1014C000DACFEAFFEE2A000EEE22EE22EE22D1D78C
:1014D000040EE15C02E2E16AE552E16EE552E7CF1B
:1014E000D9FF12000F0EC16E070EB46E936A300E54
:1014F000926E0F0E946EF19E816A80901200D9CF89
:10150000E6FFE1CFD9FF020EE1268250020B01E097
:10151000010E080DF3CF16F08250010B040DF3CF2E
:1015200015F08050200B01E0010EE824146E80506D
:10153000100B01E0010E142415241624DE6EDD6A62
:10154000DECF14F0DDCF15F014C0F3FF15C0F4FFAB
:10155000020EE15C03E200D0E16AE552E16EE55281
:10156000E7CFD9FF12008092320EE66E8AEC13F0BC
:10157000E5528084320EE66E8AEC13F0E5528094D8
:10158000320EE66E8AEC13F0E55212008082320EC3
:10159000E66E8AEC13F0E5528084320EE66E8AEC39
:1015A00013F0E5528094320EE66E8AEC13F0E552A9
:1015B0001200380E816ED7DF320EE66EE66A4DDF1E
:1015C000E552E552010E816ECEDF320EE66EE66A1E
:1015D00044DFE552E5520D0E816EC5DF320EE66E38
:1015E000E66A3BDFE552E552060E816EBCDF320E45
:1015F000E66EE66A32DFE552E5521200010E816EB8
:10160000B2DF0A0EE66EE66A28DFE552E552120006
:10161000D9CFE6FFE1CFD9FF020E816EA4DF0A0E1B
:10162000E66EE66A1ADFE552E552FD0EDBCFE6FF15
:10163000FE0EDB50280DF350E552E724E76EFE0E58
:10164000E7CFDBFFFD0EDB6AFE0EDB50F36EFD0E17
:10165000DBCFF4FFF350F45C0BE2140E816E83DFFA
:10166000320EE66E8AEC13F0E552FD0EDB2AECD763
:10167000E552E7CFD9FF1200D9CFE6FFE1CFD9FF7E
:10168000FE0EDB50816E82DF320EE66E8AEC13F0C6
:10169000E552E552E7CFD9FF1200D9CFE6FFE1CFFF
:1016A000D9FFFD0EDBCFE9FFFE0EDBCFEAFFEF50E7
:1016B0000EE0FD0EDBCFE9FFDB2AFE0EDBCFEAFFFB
:1016C00001E3DB2AEF50E66ED7DFE552EAD7E552B9
:1016D000E7CFD9FF12000201046B300E926EF00EBC
:1016E000936EEF0E006F00C281FF040E016F015177
:1016F000000821E20051FE0BE842006F00C281FFAA
:10170000050EE66EE66AA9DEE552E5528150100B41
:1017100009E08150200B06E08150400B03E081502E
:10172000800B01E10AD80201040502E1055104D051
:101730000105016FDCD7CFD71200F00E936E81CF79
:1017400003F202010315026F0F0E0015006F005126
:101750000211006F81CF03F2F00E0315026FF00E3D
:10176000025D01E0F7D7936A06D806C205F20201CE
:10177000010E046F12000201076B100E075D14E2E8
:101780000751EA6A600FE96E000EEA22EF50005D31
:1017900008E10751EA6A700FE96E000EEA22EFCF06
:1017A00006F20729076FE9D706C281FF640EE66ECD
:1017B000E66A53DEE552E55212000201086B070E9D
:1017C000085D1DE288DF0201096F0851EA6A0A0F0D
:1017D000E96E020EEA2209C2EFFF0851EA6A0A0F17
:1017E000E96E020EEA22EF50460802E108D004D06A
:1017F00009C2E6FF41DFE5520201082BE0D708519C
:10180000EA6A0A0FE96E020EEA22EF6A120002018A
:10181000086B070E085D16E20851EA6A0A0FE96EC6
:10182000020EEA22EF50E66E27DFE5520201082998
:10183000EA6A0A0FE96E020EEA22EF5001E102D0D5
:10184000082BE7D71200D9CFE6FFE1CFD9FFE65248
:10185000F250800B01E0010EDF6EF29EA69EA69C68
:10186000A684FE0EDB50A96EFD0EDB50A86E550E51
:10187000A76EAA0EA76EA682A6B2FED7A694DF50C8
:10188000E8B0F28EE8A0F29EE552E552E7CFD9FF2C
:101890001200D9CFE6FFE1CFD9FFA69CA69EFE0E8F
:1018A000DB50A96EA680A85000D0E552E7CFD9FF43
:1018B0001200D9CFE6FFE1CFD9FF120EE126DE6A92
:1018C000DD6AB6D8CC0EE66EE66AC3D8E552E552BC
:1018D000440EE66EE66ABDD8E552E552D9CFE9FF7F
:1018E000DACFEAFFEE50ED1006E11ED9F3CFDEFFAE
:1018F000F4CFDDFFF3D79CD8CC0EE66EE66AA9D80C
:10190000E552E552BE0EE66EE66AA3D8E552E55210
:101910000BD9020EF3CFDBFF030EF4CFDBFF04D9AC
:10192000040EF3CFDBFF050EF4CFDBFF040EDBCF9D
:1019300018F0050EDBCF19F018C019F0186A020E66
:10194000DB501824146E030EDB501920156E166A36
:10195000176A15AE02D016681768060E14C0DBFFB2
:10196000070E15C0DBFF080E16C0DBFF090E17C0FF
:10197000DBFF060EDBCF18F0070EDBCF19F0080EE9
:10198000DBCF1AF0090EDBCF1BF018C004F019C032
:1019900005F01AC006F01BC007F074EC0FF005C08C
:1019A00014F006C015F007C016F008C017F00A6A58
:1019B0000B6A800E0C6E410E0D6E14C005F015C042
:1019C00006F016C007F017C008F024EC10F00E0E59
:1019D00005C0DBFF0F0E06C0DBFF100E07C0DBFFEC
:1019E000110E08C0DBFFC80EE66EE66A36DDE55272
:1019F000E5520E0EDBCF14F00F0EDBCF15F0100EFC
:101A0000DBCF16F0110EDBCF17F014C004F015C0B9
:101A100005F016C006F017C007F0120EE15C03E2F5
:101A200000D0E16AE552E16EE552E7CFD9FF12003E
:101A3000926A8096010EE66EE66A0FDDE552E55287
:101A4000080E926E010EE66EE66A07DDE552E5527B
:101A50001200D9CFE6FFE1CFD9FF040EE126020E36
:101A6000DB6A030EDB6A020EDBCF14F0030EDBCF62
:101A700015F0D890155004E6080E145C000E1558A9
:101A800049E2926A8096020EE66E8AEC13F0E55205
:101A9000010EE76EFD0EDBCF14F0FE0EDBCF15F06E
:101AA000E7501416156A14C0DEFF15C0DDFFD9CF4C
:101AB000E9FFDACFEAFF010EEE1801E1ED5001E196
:101AC0008086D9CFE9FFDACFEAFFEE50ED1001E1D1
:101AD00080963C0EE66E8AEC13F0E552080E926E8C
:101AE000020EE66E8AEC13F0E552FD0EDBCF14F029
:101AF000FE0EDBCF15F0D89015321432FD0E14C057
:101B0000DBFFFE0E15C0DBFF020EDB2A030E01E336
:101B1000DB2AA9D7040EE15C02E2E16AE552E16E3C
:101B2000E552E7CFD9FF1200D9CFE6FFE1CFD9FFC9
:101B3000040EE126DE6ADD6ADECF14F0DDCF15F09B
:101B4000D890155004E6080E145C000E15584BE2B0
:101B5000926A8096020EE66E8AEC13F0E552080E49
:101B6000926EE66E8AEC13F0E552020EDBCF14F0B3
:101B7000030EDBCF15F0D89015321432020E14C0CC
:101B8000DBFF030E15C0DBFF80A610D0800EE76ED2
:101B9000020EDBCF14F0030EDBCF15F0E75014126A
:101BA000020E14C0DBFF030E15C0DBFF80B611D0A0
:101BB0007F0EE76E020EDBCF14F0030EDBCF15F0C5
:101BC000E7501416156A020E14C0DBFF030E15C091
:101BD000DBFF780EE66E8AEC13F0E552DF2A010E89
:101BE00001E3DB2AA9D7020EDBCF14F0030EDBCF13
:101BF00015F014C0F3FF15C0F4FF040EE15C03E21E
:101C000000D0E16AE552E16EE552E7CFD9FF12005C
:101C100069DCCFDC800EE66E000EE66E3EDDE5523E
:101C2000E552E66A010EE66EF3DCE552E55241DE6E
:101C300004C013F205C014F206C015F207C016F274
:101C40001C6A1D6A100E1E6E410E1F6E13C20AF032
:101C500014C20BF015C20CF016C20DF01CC005F03A
:101C60001DC006F01EC007F01FC008F077EC10F092
:101C700005C018F006C019F007C01AF008C01BF024
:101C80000A6A0B6AA00E0C6E400E0D6E18C005F0AD
:101C900019C006F01AC007F01BC008F024EC10F0C1
:101CA00005C014F006C015F007C016F008C017F004
:101CB0000A6A0B6A0C6A420E0D6E14C005F015C05C
:101CC00006F016C007F017C008F08EEC0FF005C044
:101CD00017F206C018F207C019F208C01AF280B84D
:101CE00071D013C205F014C206F015C207F016C277
:101CF00008F0E4EC10F006C01BF207C01CF21BC297
:101D000006F01CC207F05FEC0FF005C018F006C02B
:101D100019F007C01AF008C01BF018C00AF019C06B
:101D20000BF01AC00CF01BC00DF013C205F014C26A
:101D300006F015C207F016C208F08DEC0FF005C0D2
:101D400014F006C015F007C016F008C017F00A6AB4
:101D50000B6A200E0C6E410E0D6E14C005F015C0FE
:101D600006F016C007F017C008F077EC10F0E4ECAE
:101D700010F006C01DF207C01EF21DC2E6FF1EC213
:101D8000E6FF1BC2E6FF1CC2E6FF340E146E270EF0
:101D9000156E166A14C0E6FF15C0E6FF16C0E6FF12
:101DA0001F0EE66E020EE66EC6EC11F0176E090EFF
:101DB000E15E17501F0EE66E020EE66E6EDCE55217
:101DC000E55271D017C205F018C206F019C207F02B
:101DD0001AC208F0E4EC10F006C01BF207C01CF2B7
:101DE0001BC206F01CC207F05FEC0FF005C018F034
:101DF00006C019F007C01AF008C01BF018C00AF09E
:101E000019C00BF01AC00CF01BC00DF017C205F082
:101E100018C206F019C207F01AC208F08DEC0FF0D4
:101E200005C014F006C015F007C016F008C017F082
:101E30000A6A0B6A200E0C6E410E0D6E14C005F07E
:101E400015C006F016C007F017C008F077EC10F0C8
:101E5000E4EC10F006C01DF207C01EF21DC2E6FF42
:101E60001EC2E6FF1BC2E6FF1CC2E6FF2A0E146E6E
:101E7000270E156E166A14C0E6FF15C0E6FF16C0E1
:101E8000E6FF1F0EE66E020EE66EC6EC11F0176E50
:101E9000090EE15E17501F0EE66E020EE66E4DEC67
:101EA0000BF0E552E552E80EE66E030EE66E2DEC01
:0A1EB0000AF0E552E552B5D6120023
:061EBA000F9E08D00F9EF0
:101EC00007AE05D0066C071EE86A07220F8E07C012
:101ED00001F006C000F0136A126A8E0E026E036AE9
:101EE0002FEF11F00F9E0CD00F9E07AE09D0046C9F
:101EF000051E061E071EE86A0522062207220F8E0F
:101F000007C001F006C000F005C013F004C012F0D5
:101F10009E0E026E036A2FEF11F00D7E0F6A6BECBE
:101F200011F083EC11F00FB613EF11F00FA20AD0ED
:101F30000FAA03D00FBE13EF11F00FA41FEF11F083
:101F40001CEF11F00FAA05D00FAC1FEF11F01CEF22
:101F500011F00FA00AD00FA808D00FBE04D00FA414
:101F600002D028EF11F02CEF11F0126A036A0D5025
:101F7000085C116E10E305C013F006C000F007C046
:101F800001F008C010F00AC005F00BC006F00CC04C
:101F900007F00F3A09D00AC013F00BC000F00CC0D4
:101FA00001F00DC010F0116C0F9E0FBC0F8E10C011
:101FB00002F00FB05BEF11F01A0E11605BEF11F041
:101FC000026A086A0FA408D0056C061E071E081EC8
:101FD000E86A0622072208220FAC08D0136C001E04
:101FE000011E021EE86A002201220222046A115226
:101FF00007E008340732063205320432112EF9D7D1
:1020000005501326065000220750012208500222D4
:1020100004C012F00F9E02AE0BD0126C131E001EF5
:10202000011E021EE86A13220022012202220F8EE4
:1020300002A006D0D8800132003213321232102AA8
:1020400010C002F02FEF11F00F6A6BEC11F083EC6F
:1020500011F00FB613EF11F00FA205D00FBA13EF66
:1020600011F01AEF11F00FBA26EF11F00FA005D002
:102070000FB813EF11F026EF11F00FB81AEF11F0AF
:10208000036A7F0E0824026EE86A03220D50025E86
:10209000E86A035A1A0E106E086A126A136A006A16
:1020A000016A0A50055E0B50065A0C50075A000E82
:1020B000085A09E70A5005260B5006220C50072241
:1020C000000E082201D0128AD8900536063607364F
:1020D0000836D8901236133600360136102EE1D766
:1020E000075006100510D8A4128A2FEF11F00F6ABE
:1020F0006BEC11F083EC11F00FB613EF11F00FA29F
:1021000005D00FB813EF11F01AEF11F00FAA05D098
:102110000FB013EF11F01AEF11F00FB002D00FA8AB
:1021200002D026EF11F0036A0D500824026EE86A0F
:1021300003227E0E025EE86A035A126A136A006A7C
:10214000016A0C500702F4CF01F0F3CF00F00B50FE
:102150000702F3501326F4500022000E01220C5007
:102160000602F3501326F4500022000E01220A50FA
:102170000702F3501226F4501322000E002201220F
:102180000B500602F3501226F4501322000E0022C8
:1021900001220C500502F3501226F4501322000EB7
:1021A000002201220A500602F4501226000E1322C9
:1021B000002201220B500502F4501226000E1322B9
:1021C000002201222FEF11F00F6A6BEC11F00FB615
:1021D000EEEF10F00FA20ED00FB405D07F0E076EF9
:1021E000FF0E066E1FD0800E076E066A1BD0076AB0
:1021F000066A18D00FB0FBD78F0E0860EDD77E0EA1
:102200000864F5D78E0E085C05E0D89007320632D8
:10221000082AF8D70FA406D0066C071EE86A072222
:1022200007AEE5D712007F0E086EFF0E076E066E32
:10223000056E12007F0E0FBEFF0E086E02D07F0EDD
:10224000086E800E076E066A056AF3D70FAE04D0DB
:10225000800E086E076AF7D7086A076AF4D701503C
:10226000001013101210F8E003BEF0D701BE0CD01E
:1022700002500310EBE0D8901236133600360136C8
:102280000206D8A00306F2D70350D4E10228D2E018
:1022900012AE11D07F0E121402E113A00CD0132A3B
:1022A000E86A0022012207E3D880013200321332AB
:1022B000022A0228BFE00250C9E013C005F000C0A6
:1022C00006F00134076E0230086E0732089E0FBE1A
:1022D000088E19EF11F00736083602E30F840F7EDF
:1022E00006E10F80086A076A066A056A1200082874
:1022F00003E0D88007321200D890073202E10F8243
:1023000012000F8612000C360D3602E30F8C0F7E82
:1023100006E10F880D6A0C6A0B6A0A6A12000D2822
:1023200003E0D8800C321200D8900C32EAE10F8A18
:10233000120007C013F006C012F006500B02F4CFD3
:1023400005F0F3CF04F007500C02F4CF07F0F3CF01
:1023500006F00B02F3500526F4500622E86A072225
:1023600012500C02F3500526F4500622E86A0722A8
:102370000CAEBFEF11F01250065E1350075A13AEA9
:0C238000000C0B50065E0C50075A000CBD
:04238C00D9CFE6FFC0
:10239000DACFE6FFE1CFD9FFE2CFDAFFE652E6522D
:1023A000E652E652D950F90F146EFF0EDA20156E80
:1023B000020E14C0DBFF030E15C0DBFF020EDBCFE5
:1023C000E6FF030EDBCFE6FFF90EDBCFE6FFFA0EEA
:1023D000DBCFE6FFFB0EDBCFE6FFD950FC0FE66E4E
:1023E000FF0EDA20E66E32EC04F0146E070EE15CAC
:1023F00002E2E16AE552E16E1450F3CFDEFFF4CF62
:10240000DDFFFC0EDBCFE9FFFD0EDBCFEAFFEF6A5D
:10241000DECF14F0DDCF15F014C0F3FF15C0F4FFCC
:10242000040EE15C02E2E16AE552E16EE552E5CFBD
:08243000DAFFE7CFD9FF12002B
:082438002A0EF66E080EF76E85
:10244000000EF86E02010900F5502C6F0900F550DE
:102450002D6F03E12C6701D03DD00900F550276FA7
:102460000900F550286F0900F550296F090009008F
:10247000F550E96E0900F550EA6E090009000900FF
:10248000F5502A6F0900F5502B6F09000900F6CFAF
:102490002EF2F7CF2FF2F8CF30F227C2F6FF28C284
:1024A000F7FF29C2F8FF02012A5302E12B5307E08C
:1024B0000900F550EE6E2A07F8E22B07F9D72EC275
:1024C000F6FF2FC2F7FF30C2F8FF02012C07000E03
:0624D0002D5BBFD71200D6
:0A24D600D9CFE6FFDACFE6FFE1CF31
:1024E000D9FFE2CFDAFFFB0EDBCF14F0FC0EDBCF1F
:1024F00015F00001800E15141AE1FB0EDBCFE9FF89
:10250000FC0EDBCFEAFFEECFF3FFEDCFF4FFEE2AB8
:10251000000EEF22F3CFE9FFF4CFEAFFFD0EDBCF91
:10252000EFFFEF50156AF36E15C0F4FF10D0FB0EED
:10253000DB50FE0806E1FD0EDBCFE6FF7CEC13F07E
:1025400005D0FD0EDBCFE6FFA8EC13F0E552E55217
:0A255000E5CFDAFFE7CFD9FF120054
:06255A0004500902F3CF5A
:1025600000F0F4CF01F00A02F3500126000EF4202F
:10257000026E04500B02F3500226000EF420036E8C
:1025800004500C02F350032605500902F3500126B3
:10259000F4500222000E032205500A02F3500226D4
:1025A000F450032205500B02F35003260650090293
:1025B000F3500226F450032206500A02F350032679
:0A25C00007500902F3500326120031
:0625CA00FE0EE3CFE9FF65
:1025D000FF0EE3CFEAFFF36AF46AEE5203E0F34A38
:1025E000F42AFBD71200FF0EE3CFF8FFE552FF0EEF
:1025F000E3CFF7FFE552FF0EE3CFF6FFE552E66AC1
:10260000E66AE66A0900F55209E0FD0EE32A05E1F3
:10261000FE0EE32A02E1FF0EE32AF4D7FD0EE3CF1C
:1026200005F0FE0EE3CF06F0FF0EE3CF07F0120039
:10263000036A026A016A006A200EE76ED8900436C7
:10264000053606360736003601360236033609509F
:10265000005C0A5001580B5002580C50035809E313
:102660000950005E0A50015A0B50025A0C50035A8E
:08267000042AE72EE4D7120052
:08267800F36AF46AFF0EE1248D
:10268000E96EFF0EE220EA6EED6607D02F0EEF64D2
:0C26900004D03A0EEF6001D0F32A1200D3
:04269C00FF0EE350FA
:1026A000206E480E01D04C0EE76EE72EFED7E76A8B
:0C26B000E72EFED7202EF7D70000120006
:0426BC00000EF36EAB
:1026C00000EE00F0080E01D81200EA6002D0EE6AB7
:0C26D000FCD7F350E9601200EE6AFCD762
:0426DC0012EE40F0CA
:1026E00022EE40F0F86A0F9C1CEC12F0A9EC13F0FB
:0826F00008EC0EF0FBD712000C
:0826F800FF0EE350ACBA04D060
:10270000AF6AAB8EAC8A949CACA2FED7AD6EF36E72
:04271000F46A120055
:0C271400FF0EE350E84E1200000000D061
:0A27200000D000D0E82EFAD7120016
:06272A002533642E256436
:0E27300020B046002533642E256420B04300FF
:02273E00303138
:0F27400032333435363738396162636465660089
:02275000120075
:02275200120073
:0C275400EEEDEBE7DEDDDBD7BEBDBBB772
:102760007E7D7B77303132333435363738394142EC
:0A2770004344454654454D503D00DA
:00000001FF
